:0300000002057284
:0C057200787FE4F6D8FD7581160205B90B
:0F09AB00D2A2E4FF12068A12002D12026380FB13
:1005FE0000040601FF003E01020300FF0310020388
:10060E000100FF03AB03010200FF044604060005D0
:10061E00FF00F505070704FF06F306000408FF01B7
:10062E00AC07050504FF075908090906FF07BF09AE
:10063E00080806FF0824000000000000000000006B
:10064E00000000000000000000000000000000009C
:10065E00000000000000000000000000000000008C
:10066E00000000000000000000000000000000007C
:0C067E0000000000000000000000000070
:0309BA0001120027
:040973007F017E0082
:100977007D707C17D3EF9400EE94004007EF1F7053
:0D098700F31E80F0ED1D70011CED4C70E7BB
:010994002240
:10003E00E4F50E750F017510047511017B0CFA7D38
:10004E00027F01120889E4F508F509E5092403FF8A
:10005E00E4F50E750F01751004751101AB09AA08B0
:10006E007D021208890509E50970020508C3940589
:10007E00E5086480948040D3E4F508F509E5092489
:10008E0003FFE5092405FBE43508FAE4F50E750FC8
:10009E00017510047511017D031208890509E50922
:1000AE0070020508C39405E5086480948040CEE490
:1000BE00F508F509E5092403FFE5092441FBE435BC
:1000CE0008FAE4F50E750F017510047511017D0423
:1000DE001208890509E50970020508C39405E508AB
:0600EE006480948040CE06
:0100F40022E9
:10031000E4F50E750F017510047511017B0CFA7D63
:10032000027F01120889E4F508F509E5092403FFB5
:10033000E5092480FBE5083401FAE4F50E750F01A8
:100340007510047511017D021208890509E509700F
:10035000020508C39403E5086480948040CDE4F569
:1003600008F509E5092403FFE50924B6FBE435088F
:10037000FAE4F50E750F017510047511017D031275
:1003800008890509E50970020508C39402E50864B7
:1003900080948040CEE4F50E750F01751004751140
:0B03A000017B0BFA7D047F030208893B
:1003AB00E4F50E750F017510047511017B0CFA7DC8
:1003BB00037F01120889E4F508F509E5092403FF19
:1003CB00E5092480FBE5083401FAE4F50E750F010D
:1003DB007510047511017D021208890509E5097074
:1003EB00020508C39403E5086480948040CDE4F5CE
:1003FB0008F509E5092403FFE50924B6FBE43508F4
:10040B00FAE4F50E750F017510047511017D0312D9
:10041B0008890509E50970020508C39402E508641B
:10042B0080948040CEE4F50E750F017510047511A4
:0B043B00017B0BFA7D047F030208899F
:10044600E4F50E750F017510047511017B0CFA7D2C
:10045600047F01120889E4F508F509E5092403FF7C
:10046600E5092480FBE5083401FAE4F50E750F0171
:100476007510047511017D021208890509E50970D8
:10048600020508C39403E5086480948040CDE4F532
:1004960008F509E5092403FFE50924B6FBE4350858
:1004A600FAE4F50E750F017510047511017D03123E
:1004B60008890509E50970020508C39402E5086480
:1004C60080948040CEE4F50E750F01751004751109
:0B04D600017B0BFA7D047F0302088904
:1000F500E4F50E750F017510047511017B0CFA7D81
:10010500037F01120889E4F508F509E5092403FFD1
:10011500E4F50E750F01751004751101AB09AA08F8
:100125007D021208890509E50970020508C39405D1
:10013500E5086480948040D3E4F508F509E50924D1
:1001450003FFE5092405FBE43508FAE4F50E750F10
:10015500017510047511017D031208890509E5096A
:1001650070020508C39405E5086480948040CEE4D8
:10017500F508F509E5092403FFE5092441FBE43504
:1001850008FAE4F50E750F017510047511017D046B
:100195001208890509E50970020508C39405E508F3
:0601A5006480948040CE4E
:0101AB002231
:1006F300E4F50E750F017510047511017B0CFA7D7D
:10070300027F01120889750800750901C3E5099480
:100713000AE508648094805027E5092403FFE4F583
:100723000E750F01751004751101AB09AA087D023E
:1007330012088974022509F509E43508F50880CC07
:10074300E4F50E750F017510047511017B0BFA7D2D
:06075300037F0302088988
:1001AC00E4F50E750F017510047511017B0CFA7DC9
:1001BC00047F01120889E4F508F509E5092403FF19
:1001CC00E4F50E750F01751004751101AB09AA0841
:1001DC007D021208890509E50970020508C394051A
:1001EC00E5086480948040D3E4F508F509E509241A
:1001FC0003FFE5092405FBE43508FAE4F50E750F59
:10020C00017510047511017D031208890509E509B2
:10021C0070020508C39405E5086480948040CEE420
:10022C00F508F509E5092403FFE5092441FBE4354C
:10023C0008FAE4F50E750F017510047511017D04B3
:10024C001208890509E50970020508C39405E5083B
:06025C006480948040CE96
:010262002279
:10075900E4F50E750F017510047511017B0CFA7D16
:10076900037F01120889750800750901C3E5099419
:100779000AE508648094805027E5092403FFE4F51D
:100789000E750F01751004751101AB09AA087D02D8
:1007990012088974022509F509E43508F50880CCA1
:1007A900E4F50E750F017510047511017B0BFA7DC7
:0607B900037F0302088922
:1007BF00E4F50E750F017510047511017B0CFA7DB0
:1007CF00027F01120889E4F508F509C3E509940AC7
:1007DF00E508648094805027E5092403FFE4F50EB3
:1007EF00750F01751004751101AB09AA087D02126E
:1007FF00088974022509F509E43508F50880CCE469
:10080F00F50E750F017510047511017B0BFA7D0341
:05081F007F03020889BF
:10082400E4F50E750F017510047511017B0CFA7D4A
:10083400037F01120889E4F508F509C3E509940A60
:10084400E508648094805027E5092403FFE4F50E4D
:10085400750F01751004751101AB09AA087D021208
:10086400088974022509F509E43508F50880CCE403
:10087400F50E750F017510047511017B0BFA7D03DC
:050884007F030208895A
:1002630020B33112097320B32B30B3FD7D027F011C
:1002730012094E7D037F0112094E7D047F0112098D
:100283004EE51275F007A42400F582E43406F583E5
:10029300E493F51220B53112097320B52B30B5FD67
:1002A3007D027F0112094E7D037F0112094E7D04F9
:1002B3007F0112094EE51275F007A424FFF582E4CD
:1002C3003405F583E493F51220B21F12097320B2AB
:1002D3001930B2FD12002DE51275F007A42401F5C3
:1002E30082E43406F583E493F512E51275F007A46E
:1002F3002402F582E43406F583E493FB740193FA54
:0D030300740293F98B138A14F51502051787
:0309BD0001160020
:0F08E6001208F5D2A11208F5C2A11208F5D2A18D
:1008F500E4FDFCC3ED9FEC9E50257B307A00900013
:100905000AE582158270021583E582458370F2EB54
:0F0915001B70011AEB4A70E60DBD00010C80D477
:0109240022B0
:10000300ED131354032480FCEDC43354602EAF046A
:06001300FE120019AF0609
:10001900EFC2A17F08C2A2A2E092A3D2A2C313DFBA
:03002900F4D2A16D
:01002C0022B1
:02094E00AE07F2
:10095000EED39417501CED940B50171200037F88B0
:10096000120019E4FF1200197F901200197F3E1245
:0209700000196C
:010972002262
:02099500AB07AE
:10099700EBD3940B500DE4FAAF02AD0312094E0AE4
:0309A700BA18F586
:0109AA00222A
:0B002D00E4F9AF0112099509B90CF7C6
:0100380022A5
:02092500AE071B
:10092700EE131354032484FDEEC433546004AF055F
:100937001200137F88120019E4FF1200197F90122A
:070947000019E4FF02001992
:02088900AE07B8
:10088B00EED394175054ED940B504F120003E50E1A
:10089B0044B0FF120019ED4420FF120019E516B405
:1008AB000406751007E4F50FE510C45470450FFEF0
:1008BB00E5114488FF1200147C007D80AF03AE026B
:1008CB001204E1EF2490FF120019AE02AF037C007B
:0A08DB007D801204E1AF0512001940
:0108E50022F0
:02068A00A907BE
:10068C00C2A17F0A7E001208E6C2A11208E67FA072
:10069C00120019E4FF1200197FAD1200197F10121D
:1006AC0000197FBC1200197F201200197FC01200A4
:1006BC00197F0A1200197FC81200197F2012001925
:1006CC007FD1120019E94438FF120019E51644A233
:1006DC00FF1200197F2B120019E4FCAF041209253C
:0706EC000CBC0BF702002D0E
:10057E000209ABE493A3F8E493A34003F68001F2DF
:10058E0008DFF48029E493A3F85407240CC8C3337E
:10059E00C4540F4420C8834004F456800146F6DF4D
:1005AE00E4800B01020408102040809009BAE47E1A
:1005BE00019360BCA3FF543F30E509541FFEE49342
:1005CE00A360010ECF54C025E060A840B8E493A309
:1005DE00FAE493A3F8E493A3C8C582C8CAC583CA34
:1005EE00F0A3C8C582C8CAC583CADFE9DEE780BEEC
:0109C0000036
:1004E100C2D5EC30E709B2D5E4C39DFDE49CFCEE36
:1004F10030E715B2D5E4C39FFFE49EFE12051DC38C
:10050100E49DFDE49CFC800312051D30D507C3E486
:060511009FFFE49EFE22A4
:060517008A838982E4736F
:10051D00BC000BBE0029EF8DF084FFADF022E4CCC2
:10052D00F875F008EF2FFFEE33FEEC33FCEE9DEC8B
:10053D00984005FCEE9DFE0FD5F0E9E4CEFD22EDD1
:10054D00F8F5F0EE8420D21CFEADF075F008EF2F1B
:10055D00FFED33FD4007985006D5F0F222C398FD0C
:05056D000FD5F0EA22A9
:00000001FF
